:03000000023B8937
:0C3B890078FFE4F6D8FD758167023BD0A0
:101430000A53746172743A20004950436F6E6E65AE
:1014400063745245510A004950436F6E6E65637470
:10145000003E432C562C43432CC0E4E0EFF2E5F071
:1014600020D1E8EDEAEEEC49500A003E432C4D4114
:10147000432C25303262583A25303262583A2530B2
:101480003262583A25303262583A25303262583A40
:1014900025303262582C4D414320E0E4F0E5F10A5A
:1014A000003E432C5645522C20332E3120EEF220A4
:1014B00025732025732CC2E5F0F1E8FF2049502068
:1014C000ECEEE4F3EBFF0A004E6F7620303320326F
:1014D0003030370030383A35323A3433003E432C1E
:1014E0004C442C50524F473A2020202020202020CE
:1014F00020202020202020202020202020202020EC
:1015000020202020202020202020202020202020DB
:1015100020202020202020202020202020202020CB
:10152000202020202020202020202020202CC4E04B
:10153000F2E020EFF0EEF8E8E2EAE828F4E0E9EB88
:10154000290A003E2A2C312CCEF1EDEEE2EDFBE52E
:1015500020EFE0F0E0ECE5F2F0FB20F1E5F2E5E26F
:10156000EEE3EE20E8EDF2E5F0F4E5E9F1E00A0063
:101570003E412C4130312C2562752E2562752E2579
:1015800062752E2562752C495020E0E4F0E5F120CB
:10159000E0E4E0EFF2E5F0E00A003E412C413032B9
:1015A0002C2562752E2562752E2562752E25627595
:1015B0002C495020E0E4F0E5F120EEF1ED2E20F191
:1015C000E5F0E2E5F0E00A003E412C4130332C2505
:1015D00062752E2562752E2562752E2562752C4941
:1015E0005020E0E4F0E5F120F0E5E72E20F1E5F011
:1015F000E2E5F0E00A003E412C4130342C256275D2
:101600002E2562752E2562752E2562752CCCE0F193
:10161000EAE020F1E5F2E80A003E412C4130352CA9
:101620002562752E2562752E2562752E2562752C14
:10163000D8EBFEE70A003E532C4130362C2562756C
:101640002CC2F0E5ECFF20EEE6E8E42E20EAE2E82A
:10165000F2E0EDF6E8E820282A3130ECF1290A0022
:101660003E2A2C312CC4EEEF2E20EFE0F0E0ECE52A
:10167000F2F0FB20F1E5F2E5E2EEE3EE20E8EDF238
:10168000E5F0F4E5E9F1E00A003E422C5330312C5C
:101690002562752CC6E4E0F2FC20E7E0EFF0EEF105
:1016A000E020F1EEE5E4E8EDE5EDE8FF20EEF220E4
:1016B000F1E5F0E2E5F0E00A003E422C5330322C36
:1016C0002562752CCEE1ECE5ED20F120F1E5F0E2AC
:1016D000E5F0EEEC20E1E5E720EAE2E8F2E0EDF605
:1016E000E8E90A003E422C5330332C2562752CCF9A
:1016F000E5F0E5E7E0EFF3F1EA20EFF0E820EFEEC8
:10170000F2E5F0E520F1E2FFE7E820F120F1E5F075
:10171000E2E5F0EEEC0A003E422C5330342C256218
:10172000752CCDE5F220EFE5F0E5E4E0F7E820E404
:10173000E8E0E3EDEEF1F2E8EAE820E220F1E5F09E
:10174000E2E5F00A003E422C5330352C2562752C20
:10175000CAE0EDE0EB20F8E8F0EEEAEEE2E5F8E0D2
:10176000F2E5EBFCEDEEE3EE20EEE1ECE5EDE00A78
:10177000003E532C5330362C2530326258253032FF
:101780006258253032625825303262582530326234
:101790005825303262582C4D414320E0E4F0E5F109
:1017A00020F8E8F0EEEAEEE2E5F8E0F2E5EBFCED39
:1017B000EEE3EE20EEE1ECE5EDE00A003E454E44BE
:1017C0000A0044756D7058202020202030302030D1
:1017D0003120303220303320303420303520303644
:1017E000203037203038203039203041203042201E
:1017F00030432030442030452030460A003A200053
:101800000A0044756D7044202020202030302030A4
:101810003120303220303320303420303520303603
:1018200020303720303820303920304120304220DD
:1018300030432030442030452030460A0045727243
:10184000206B657900526420656570726F6D0A00C7
:101850005264204D454D0A00526420436F64650A6E
:101860000044656275674950204F4E0A0044656226
:1018700075674950204F46460A00446562756755B2
:10188000736572204F6E0A00446562756755736513
:1018900072204F46460A0044656275674D736720A3
:1018A0004F6E0A0044656275674D7367204F464668
:1018B0000A00436F6E666967206C6F636B210A00D4
:1018C000577220656570726F6D0A002053617665EE
:1018D00020656570726F6D210A00457272204D415E
:1018E0004321004C6F61643E3E002A003C41303190
:1018F0003D003C4130323D003C4130333D003C41F5
:1019000030343D003C4130353D003C4130363D00F7
:101910004E4F4950004C494E4B434F4E5452005489
:1019200052415353004652004E4F4C494E4B0049D2
:101930004E49004E4F4449414700003C21003C5372
:1019400030313D003C5330323D003C5330333D009C
:101950003C5330343D003C5330353D003C53303631
:101960003D00FF1910FF1915FF191FFF1925FF1959
:0A19700028FF192FFF1933FF193A61
:06453500010B000109006A
:10452100C2AFC28E438910758BFF758DB7D2ABD2E6
:044531008ED2AF2255
:03001B00023A5F47
:103A5F00C0E0C083C082C0D0C2AFC28E758BFF756D
:103A6F008DB720060675A61E75A6E10509D202E5DB
:103A7F000B6002050BE50AD394014002150A050EEF
:103A8F00E50E540F7050D20DE50E543F701AD20050
:103A9F0090668DE0601204F0E0D394B4400A9080F9
:103AAF00007480F0C2AF80FE906688E0600204F080
:103ABF00906104E0600214F090668EE0D3940140B0
:103ACF0003E014F0300502050CE50DD394644004B7
:103ADF00D2068002050DE508D3940140021508D2E5
:0C3AEF008ED2AFD0D0D082D083D0E03295
:10088100C291C290D2B5C20A7D027C007F07124498
:10089100B58F49E549646060097D017F6012446D4F
:1008A100D20AE4FDFC7F0B1244B58F49E54930E6DD
:1008B100097D04E4FF124491D20A7D017C007F0787
:1008C1001244B58F49E5497008FD7FFF12446DD28E
:1008D1000A300A03126000C2AFC288C2A8C2AA7558
:1008E1008900123EA5906341E0B4FA09A3E064CE09
:1008F1007003020981E4F54974392549F582E4342C
:1009010063F583E4F00549E549B443EC9063417430
:10091100FAF0A374CEF0A374CCF0906347740AF09C
:10092100E4A3F0A304F0A3F090634C7403F0A37468
:10093100CCF090633D74FFF0A3F0A3F0E4A3F0903A
:1009410063587405F0E4F549E5492401FFE433FEF9
:1009510074392549F582E43463F583E0FD124508D5
:100961000549E549C3944340DFE4F5A775A61E7523
:10097100A6E1907FF0F0A3F09080007480F080FEFB
:10098100D2AF90634C7403F0A374CCF0E490634B4A
:10099100F0123640EF6003122AD9C2B5123C15C2DB
:1009A100061242F7906358E0C3940350037403F0B6
:1009B100D20AC20CC20BD293200A077E147F3012D6
:1009C1003726E4906578F0124521C2AFA37408F090
:1009D1009062B77424F0E4A3F0906341E09062B9AF
:1009E100F0906342E09062BAF0906343E09062BBA2
:1009F100F0906344E09062BCF0906345E09062BD8A
:100A0100F0906346E09062BEF0750A01E490657A69
:100A1100F0C207C208D2AF75A70775A61E75A6E179
:100A2100200A18AF49FE7D03123807E4FF1239B5D9
:100A31007E637F78E4FB7D011238E190668DE06092
:100A4100037401F0E4906104F0A37455F0A3748180
:100A5100F0E4F50CE4F50D906104E0700312197AED
:100A610090668EE0B401119080007410F0E49066FD
:100A71008EF0D20AD20BD20C908008E0F54930E416
:100A810005D2077410F0E54930E508D209908008D5
:100A91007420F0E54930E608D2089080087440F0EF
:100AA100E50CD394034023908002E4F0908001F0A0
:100AB100908000F0E50CD39406400FE4F50CC203DE
:100AC10090657AF0750A011242F79080A0E07003F8
:100AD100123F9E9080B8E070031240189080D0E0E1
:100AE10070031241D7908000E07013300710123567
:100AF1003C906334EFF0D3940040031200269080C1
:100B010002E07006908000E06005D205020A55C23D
:100B110005E4F50C906104E06003020A5530091206
:100B2100123197906334EFF0D394004005E0FF1247
:100B31000022200803020CB4123022906334EFF03B
:100B41007003020A55906378E054BF247F7003025A
:100B51000C17147003020BEF24026003020C4A20ED
:100B61000A077E147F39123726300E7920037690DA
:100B71006350E07006906354E0605B906684E0FF30
:100B8100906350E0B50724906685E0FE906351E0E4
:100B9100B50618906686E0FE906352E0B5060C90AB
:100BA1006687E0FE906353E06E602B906354E06FC4
:100BB1007033906685E0FF906355E0B50727906636
:100BC10086E0FF906356E0B5071B906687E0FF90D3
:100BD1006357E0B5070F90657A7401F012453F75D0
:100BE1000A01020CB490668474FFF0020CB49066A2
:100BF1008DE060037401F090667CE0FF90637AE021
:100C01006F6003020CB490667CE004F0E4F50A9096
:100C11006578F0020CB4300303020CB4906347E032
:100C21007003020A5512453DD203E4F50A90657836
:100C3100F090668804F0E490667BF0A3F0200A73DC
:100C41007E147F47123726806A90668DE0600374B8
:100C510001F0300352906378E020E74B90637AE033
:100C6100FF90667BE0FE6F600D906683E07007EE9B
:100C7100146F703F801390667BE004F0906334E062
:100C8100FFD39404400312453E9060007482F0A3A8
:100C91007401F090637AE0906002F07E607F007DE5
:100CA10003123F23020A55300E0920030690668481
:100CB10074FFF0200303020D69E50A706B123AFB21
:100CC100EF60207E647F78906479E02404FD123F18
:100CD10023906683E06003020A55906358E0F50AA9
:100CE100020A55906688E0D3943C403C906683E0CC
:100CF100703690668804F09062B6E0702B12453C25
:100D0100E4906478F0A37412F090667CE090647AC9
:100D1100F0A374FDF090610763A20190647C63A26B
:100D2100017F12122DA7809B12001EEF60159060AB
:100D3100007483F0E4A3F07E607F007D02123F2304
:100D4100020A55E50A64016003020A55906578E0DC
:100D510004F0E0C394055003020CC4C203E490659F
:100D61007AF012453F020A55E50A64016003020A5E
:100D71005590657AE014604024FE603C14700302D3
:100D81000E5124046003020A55E4F50C200E139061
:100D9100657A7404F0906578E05401F0750A0102F7
:100DA1000A55E490657AF090657804F0750AC89068
:100DB100668474FFF0020A55906684E07003020EA7
:100DC100409064787480F090647A7401F0E4A3F048
:100DD100A304F0A37430F0A3747BF0E4F549747FAD
:100DE1002549F582E43464F583747DF074802549E6
:100DF100F582E43464F583E4F0E5492407906479ED
:100E0100F07C667D8490634CE0FAA3E0FB7F0212E4
:100E11003D217E647F78E5492409FD123F239066D8
:100E210083E0601B12453DD203E4F50A906578F03A
:100E310090668804F0E490667BF0A3F0020A559076
:100E4100657A7404F0906358E02432F50A020A5579
:100E51009080027410F0750A03906578E06401FFD8
:100E6100F090657A7401F0EF7019906354E06013AB
:100E7100FCA3E0FDA3E0FEA3E0FF906684122741FE
:100E8100020A55906350E0FCA3E0FDA3E0FEA3E05D
:0C0E9100FF906684122741020A5580FE83
:010E9D002232
:10002600906379E0B444047F0180027F0090637896
:10003600E0B447047E0180027E00EE5F604A906372
:1000460041E090637AF0906342E090637BF09063C6
:1000560043E090637CF0906344E090637DF09063AE
:1000660045E090637EF0906346E090637FF0906396
:10007600797452F09062B063A2019080A863A201E5
:100086007F06122DA7020877906334E0C3940850C8
:1000960003020880906341E0FF90637AE06F60039B
:1000A600020880906342E0FF90637BE06F6003028A
:1000B6000880906343E0FF90637CE06F6003020872
:1000C60080906344E0FF90637DE06F6003020880E8
:1000D600906345E0FF90637EE06F600302088090C6
:1000E6006346E0FF90637FE06F60030208809063E1
:1000F60079E0B444159062B0E0B4FF0E63A20190BB
:1001060080A863A2017F06122DA790668DE060038A
:100116007401F090668E7464F09063797452F09076
:100126006378E0646D60030202A37BFF7A14795161
:100136001222DF7BFF7A14796B906341E0F552A3BC
:10014600E0F553A3E0F554A3E0F555A3E0F556A377
:10015600E0F5571222DF7552FF7553147554C875B2
:1001660055FF7556147557D47BFF7A1479A1122260
:10017600DF7BFF7A1479DD1222DF7BFF7A15794364
:100186001222DF7BFF7A157970906347E0F552A360
:10019600E0F553A3E0F554A3E0F5551222DF7BFF0B
:1001A6007A15799A906350E0F552A3E0F553A3E0EF
:1001B600F554A3E0F5551222DF7BFF7A1579C89036
:1001C6006354E0F552A3E0F553A3E0F554A3E0F53C
:1001D600551222DF7BFF7A1579F690633DE0F552E2
:1001E600A3E0F553A3E0F554A3E0F5551222DF7B17
:1001F600FF7A167919906339E0F552A3E0F553A317
:10020600E0F554A3E0F5551222DF7BFF7A16793626
:10021600906358E0F5521222DF7BFF7A167960125E
:1002260022DF7BFF7A167989A20EE433F552122279
:10023600DF7BFF7A1679B9906683E0F5521222DFEA
:100246007BFF7A1679E490668DE0F5521222DF7B09
:10025600FF7A1779179062B6E0F5521222DF7BFF1C
:100266007A177945A201E433F5521222DF7BFF7A31
:1002760017797190667DE0F552A3E0F553A3E0F59A
:1002860054A3E0F555A3E0F556A3E0F5571222DF97
:100296001232FD7BFF7A1779BC1222DF2290637837
:1002A600E0644C70527E177FC2123726906380E05E
:1002B600F54AA3E0F54BE4F54C7D03AF4BAE4A128D
:1002C60038077E177FFD123726AE4AAF4BE4FB7D1B
:1002D600101238E17E187F001237267410254BF570
:1002E6004BE4354AF54A054CE54CC3941040CA7EAA
:1002F600187F0012372622906378E0646C705CF5F4
:100306004E7E187F02123726E4F54DAF4E7E007DF5
:10031600031238077E177FFD123726E4F54CA84EE8
:10032600E6FF7482254CF582E43463F583EFF0052D
:100336004E054CE54CB410E67E637F82E4FB7D10EF
:100346001238E17E187F00123726054DE54DC3941D
:100356000840B87E187F0012372622906378E06442
:100366004B7061F54C746A254CF582E43463F58371
:10037600E06032746A254CF582E43463F583E0F478
:100386006023746A254CF582E43463F583E0FF74D8
:1003960080254CF582E43463F583E0B50710054CFF
:1003A600E54CB408C09061047432F002087790639B
:1003B600787421F0300A030208777E187F3D1237E1
:1003C60026020877906378E0B4521A200A077E184E
:1003D6007F451237269063787472F07E637F787D4E
:1003E60008123DA522906378E064497045200A070B
:1003F6007E187F50123726906380E0F54AA3E0F519
:100406004BE4F54C854B82854A83E0FF7482254C8C
:10041600F582E43463F583EFF0054BE54B70020596
:100426004A054CE54CB480DC7E637F787D8A123DBC
:10043600A522906378E064437079A3E06452704625
:10044600200A077E187F58123726906380E0F54A07
:10045600A3E0F54BE4F54C854B82854A83E493FF94
:100466007482254CF582E43463F583EFF0054BE5A1
:100476004B7002054A054CE54CB480DB7E637F7801
:100486007D8A123DA522906379E0645760030208D5
:1004960080906380E0F54AA3E0F54B7482254CF525
:1004A60082E43463AD82FC7B80AF4BAE4A124413C8
:1004B600020877906378E06444600302054A90631B
:1004C60080E0FF64447003020877EFB4310CC20A7F
:1004D6007E187F61123726020877906380E0B43079
:1004E6000CD20A7E187F6D12372602087790638039
:1004F600E0B4320CD20B7E187F7A123726020877C8
:10050600906380E0B4330CC20B7E187F88123726C6
:10051600020877906380E0B4340CD20C7E187F9783
:10052600123726020877906380E0B4350CC20C7E41
:10053600187FA4123726020877906380E0FF120026
:1005460021020877906104E07013200A077E187F65
:10055600B21237269063787421F00208779061040E
:100566007432F0906378E0FFB4510A908000748092
:10057600F0C2AF80FEEF64577045200A077E187FF1
:10058600C0123726906381E0906334F0E4F54C9016
:100596006334E0FFE54CC39F40030208777482256D
:1005A6004CF582E43463F583E0FF906380E0254CEC
:1005B60024AFF582E43461F583EFF0054C80D090EA
:1005C6006378E064536003020679200A077E187F89
:1005D600CB123726906341E0FF9061B8E06F703C24
:1005E600906342E0FF9061B9E06F7030906343E042
:1005F600FF9061BAE0B50724906344E0FF9061BBC9
:10060600E0B50718906345E0FF9061BCE0B5070CC4
:10061600906346E0FF9061BDE06F6016906378746A
:1006260021F0300A030208777E187FDA1237260295
:100636000877E4F54CE4F50DAF4CFE74AF254CF5A8
:1006460082E43461F583E0FD124508054CE54CC3B0
:1006560094FE40E19080007480F0C2AFE4907FF099
:10066600F0A3F0907FFD74AAF0A374FFF0A3745575
:10067600F080FE906378E0644F704C906380E0F504
:100686004AA3E0F54BE54B454A700A200A077E1857
:100696007FE3123726200A077E187FEA123726E400
:1006A600F54C7482254CF582E43463F583E0854B82
:1006B60082854A83F0054BE54B7002054A054CE5F9
:1006C6004CB480DE020877906378E0FFB44527904B
:1006D60080007480F0906380E0FDA3E0907FF0CD11
:1006E600F0A3EDF0C2AF907FFD74AAF0A374FFF003
:1006F600A37455F080FEEF6465600302087790638B
:1007060080E0FFA3E0907FF0CFF0A3EFF0E4F54A9E
:10071600F54BD3907FF1E0954B907FF0E0954A4002
:1007260020E4F50D254BFFE54A3401FE854B828515
:100736004A83E0FD124508054BE54B7002054A80E9
:10074600D17E187FEC123C9CEF4E60201200039085
:100756006347EFF0120003906348EFF01200039036
:100766006349EFF012000390634AEFF07E187FF2C0
:10077600123C9CEF4E6020120003906350EFF01283
:100786000003906351EFF0120003906352EFF012F2
:100796000003906353EFF07E187FF8123C9CEF4EF7
:1007A6006020120003906354EFF01200039063552B
:1007B600EFF0120003906356EFF0120003906357B8
:1007C600EFF07E187FFE123C9CEF4E602012000375
:1007D60090633DEFF012000390633EEFF0120003CA
:1007E60090633FEFF0120003906340EFF07E197FB5
:1007F60004123C9CEF4E6020120003906339EFF028
:1008060012000390633AEFF012000390633BEFF09F
:1008160012000390633CEFF07E197F0A123C9CEFB6
:100826004E600812429A906358EFF0E4F54CE4F5F6
:100836000DE54C2401FFE433FE7439254CF582E4C2
:100846003463F583E0FD124508054CE54CC394433B
:1008560040DC9080007480F0C2AFE4907FF0F0A39B
:10086600F0907FFD74AAF0A374FFF0A37455F08096
:0A087600FE7E637F787D08123DA529
:010880002255
:1043DB00AE07EEC39430400BEED394395005EE2468
:1043EB00D0FF22EEC39461400BEED394665005EEE2
:1043FB0024A9FF22EEC39441400BEED39446500503
:08440B00EE24C9FF22AF0622D6
:1044EE009062AFE004F070069062AEE004F090626D
:0A44FE00AEE0FEA3E0FF1244D2225C
:100003001244EE1243DBEFC454F0FEC0061244EE7A
:080013001243DBD0E02FFF22B5
:10429A00E4906C5BF01244EE906C5CEFF0C39430E7
:1042AA004018E0FFD394395011906C5BE02407F575
:1042BA0082E43461F583EFF08011906C5BE02407AF
:1042CA00F582E43461F583E4F0800C906C5BE004E1
:1042DA00F0E0D3940840BE7552007553007554003F
:0C42EA00E4F5557B017A617907122E7E05
:0142F60022A5
:043C9C008E4F8F5068
:103CA0009062AEE4F0A374FFF01244EEEF606EF4A5
:103CB000606B855082854F83E493B507EC755101A5
:103CC000E5502551F582E4354FF583E49360259066
:103CD00062AFE02551FF9062AEE03400FE1244D2A4
:103CE000E5502551F582E4354FF583E493B507049B
:103CF000055180CCE5502551F582E4354FF583E43C
:103D00009370A6E55124FFFFE434FFFE9062AFE01C
:103D10002FF09062AEE03EF07E007F0122E4FEFFD5
:013D20002280
:103640007E197F3B123C9CEF4E70037F01227E1956
:103650007F3E123C9CEF4E600C1244EEEF24D024CF
:10366000FF920E8002D20E7E197F44123C9CEF4ED8
:10367000600C1244EEEF24D0906683F08005E49055
:103680006683F07E197F4A123C9CEF4E600C124418
:10369000EEEF24D090668DF08005E490668DF07E8C
:1036A000197F50123C9CEF4E600C1244EEEF24D078
:1036B0009062B6F08005E49062B6F07E197F5612F3
:1036C0003C9CEF4E600C1244EEEF24D024FF92019C
:1036D0008002C20190634163A20190667D63A201F2
:1036E0007F06122DA730013B7E197F5C123C9CEFB8
:1036F0004E603012000390667DEFF012000390667A
:103700007EEFF012000390667FEFF01200039066E8
:1037100080EFF0120003906681EFF01200039066D4
:0637200082EFF07F0022A1
:102AD900C201E490668DF0D20EC204906683F09034
:102AE90062B6F090634163A20190667D63A2017FA3
:102AF90006122DA7E4F54AE54A75F003A42462F508
:102B090082E43419F583E493FB740193FA74029314
:102B1900F91225D97003022CCBE4F54BF54CFD7461
:102B29002F2DF582E43461F583E0FF7003022CC692
:102B3900E54A75F003A42462F582E43419F583E4C7
:102B490093FB740193FA740293F9854B82758300A0
:102B59001225F2FEEFB50608754C01054B022CC291
:102B6900E54C7003022CC2EE6003022CBDE54A2439
:102B7900FE6028147003022CA5147003022CA914FA
:102B89007003022CB1147003022CB52405600302F2
:102B99002CC690668D7401F0022CC6D201742F2DBB
:102BA900F582E43461F583E0FF642D7003022CC6DD
:102BB9001243DBEFC454F0FC74302DF582E4346128
:102BC900F583E0FF1243DBEF2C90667DF074312D25
:102BD900F582E43461F583E0FF1243DBEFC454F07E
:102BE900FC74322DF582E43461F583E0FF1243DB96
:102BF900EF2C90667EF074332DF582E43461F58311
:102C0900E0FF1243DBEFC454F0FC74342DF582E489
:102C19003461F583E0FF1243DBEF2C90667FF0749B
:102C2900352DF582E43461F583E0FF1243DBEFC40F
:102C390054F0FC74362DF582E43461F583E0FF121B
:102C490043DBEF2C906680F074372DF582E4346114
:102C5900F583E0FF1243DBEFC454F0FC74382DF523
:102C690082E43461F583E0FF1243DBEF2C90668147
:102C7900F074392DF582E43461F583E0FF1243DB0A
:102C8900EFC454F0FC743A2DF582E43461F583E025
:102C9900FF1243DBEF2C906682F08021D204801D65
:102CA9009066837401F08015C20E80119062B6742B
:102CB90001F08009E4F54CF54B0D022B28054A0279
:022CC9002B00DE
:012CCB0022E6
:10435000906579E0C3947C503D906579E0FE04F06F
:1043600074B72EF582E43462F583EFF0BF0A27902C
:104370006579E0FF04F074B72FF582E43462F583C9
:10438000E4F0906579E0FF123E279065797408F0BB
:074390009062B8E004F02286
:1042F7009080007480F090633963A201F583F582A2
:1043070063A2017F08122DA790634163A2019080E9
:104317008863A2017F0A122DA7908092E4F0A3740C
:1043270032F0A37401F090634BE0FF9080B1F090FE
:1043370080E1EFF09080957455F0A3F090800074C1
:0943470001F09080097470F0226D
:103F9E00908009E04410F09080A0E0706C9080A1B9
:103FAE007482F09080A874FFF0A3F0A3F0A3F07FCA
:103FBE00039080AEEFF07FCBA3EFF07F039080AC49
:103FCE00EFF0A374CBF09080007402F0906C4F125F
:103FDE00274D00000000906C4FE0908040F0906CF8
:103FEE0050E0908041F0906C51E0908042F0906CE7
:103FFE0052E0908043F0A3E4F0A3F0A3F0A3F0907E
:09400E008018F0A3F0A3F0A3F068
:014017002286
:1041D700908009E04440F09080D17482F090634C65
:1041E700E0FF9080DEF090634DE0FF9080DFF0907D
:1041F70080027402F0906C5312274D00000000906B
:104207006C53E0908058F0906C54E0908059F09097
:104217006C55E090805AF0906C56E090805BF0A36C
:10422700E4F0A3F0A3F0A3F0908030F0A3F0A3F0A4
:02423700A3F0F2
:014239002262
:10401800908009E04420F09080B8E0706C9080B9FE
:104028007482F07F039080C6EFF07FCDA3EFF07F1E
:10403800039080C4EFF0A374CDF09080C074FFF0BB
:10404800A3F0A3F0A3F09080017402F0906C5712D3
:10405800274D00000000906C53E090804CF0906C6D
:1040680054E090804DF0906C55E090804EF0906C4C
:1040780056E090804FF0A3E4F0A3F0A3F0A3F090F3
:094088008024F0A3F0A3F0A3F0E2
:01409100220C
:103D21008C4A8D4BA907EAFDE975F018A424ACFF74
:103D3100E5F034808F82F583EDF0EBFDE975F01845
:103D4100A4FFAEF024ACFBEE34808B82F583A3EDAF
:103D5100F0854B828C83E0FDEF24A8FFEE3480FEDA
:103D61008F82F583EDF0854B828C83A3E08F828E69
:103D710083A3F0854B82854A83A3A3E0FDE975F017
:103D810018A424A8FFE5F03480FE8F82F583A3A355
:103D9100EDF0854B828C83A3A3A3E08F828E83A356
:043DA100A3A3F022C6
:063DA5008D4FAB07AA06DA
:103DAB00906C4FE0FCA3E0FDA3E0FEA3E0F5538E87
:103DBB00528D518C50AE02AF038E838F8263A20162
:103DCB00E552540744C0F58385538263A201AF4F7C
:103DDB00122E10908000E020E5F9E4FCFDFEE55387
:103DEB00254FF553EE3552F552ED3551F551EC3576
:103DFB0050F550908040E550F0A3E551F0A3E5520B
:103E0B00F0A3E553F09080007420F0AF53AE52ADA9
:0B3E1B0051AC50906C4F122741AF4F8C
:013E26002279
:063F23008D4AAB07AA065F
:103F2900906C53E0FCA3E0FDA3E0FEA3E0F54E8E08
:103F39004D8D4C8C4BAE02AF038E838F8263A201F1
:103F4900E54D540744D0F583854E8263A201AF4AFB
:103F5900122E10E4FCFDFEE54E254AF54EEE354DD8
:103F6900F54DED354CF54CEC354BF54B908058E55E
:103F79004BF0A3E54CF0A3E54DF0A3E54EF090809E
:103F8900027420F0AF4EAE4DAD4CAC4B906C531259
:043F99002741AF4AC3
:013F9D002201
:0239B5008F4A37
:1039B700908001E030E5037F0022906C57E0FCA384
:1039C700E0FDA3E0FEA3E0F54E8E4D8D4C8C4B90B1
:1039D700667D63A201E54D540744C8F583854E8291
:1039E70063A2017F06122E26E54E2406F54EE43526
:1039F7004DF54DE4354CF54CE4354BF54B90657B77
:103A070063A201E54D540744C8F583854E8263A23E
:103A170001AF4A122E26E4FCFDFEE54E254AF54E7F
:103A2700EE354DF54DED354CF54CEC354BF54B90F2
:103A3700804CE54BF0A3E54CF0A3E54DF0A3E54E34
:103A4700F09080017420F0AF4EAE4DAD4CAC4B9072
:073A57006C57122741AF4A32
:013A5E002245
:10353C009081E0E0F54A054A054A054A054A054AE4
:10354C00054A054A054A054A054A908010E0F54DA2
:10355C00A3E0F54EA3E0F54FA3E0F5509081E1E038
:10356C00F54A054A054A054A054A054A054A054AE7
:10357C00054A054A054A908014E0F551A3E0F5523E
:10358C00A3E0F553A3E0F554E553B54F08E554B566
:10359C0050037F0022E4F54AE553540744E0F583D9
:1035AC0085548263A20190637863A2017F08122E76
:1035BC003E90637A63A2019062B063A2017F06120F
:1035CC002DA7906378E0F54BA3E0F54CE4F54A9019
:1035DC006378E0702AA3E024F8F54AE553540744D5
:1035EC00E0F58385548274082582F582E43583F5F1
:1035FC008363A20190637863A201AF4A122E3EAEA0
:10360C004BE4FCFDE554254CF554E5533EF553EDE8
:10361C003552F552EC3551F551908014E551F0A32B
:10362C00E552F0A3E553F0A3E554F090800074400C
:03363C00F0AF4AA2
:01363F002268
:103022009081E6E0F54A054A054A054A054A054AFD
:10303200054A054A054A054A054A908028E0F54DA9
:10304200A3E0F54EA3E0F54FA3E0F5509081E7E051
:10305200F54A054A054A054A054A054A054A054A06
:10306200054A054A054A90802CE0F551A3E0F55245
:10307200A3E0F553A3E0F554E4F54AE553B54F0A4E
:10308200E554B55005C20802317CE553540744F0BB
:10309200F58385548263A20190637863A2017F085D
:1030A200122E3E906378E0F54BA3E0F54CE54C45DB
:1030B2004B70099080027410F07F0022906684E0C9
:1030C200FFF4602D90637AE06F7076906685E0FF82
:1030D20090637BE06F706A906686E0FF90637CE0AD
:1030E2006F705E906687E0FF90637DE06F60228084
:1030F2005090637AE0906684F090637BE0906685FE
:10310200F090637CE0906686F090637DE090668745
:10311200F0906378E0702AA3E024F8F54AE553546E
:103122000744F0F58385548274082582F582E435DC
:1031320083F58363A20190637863A201AF4A122EE2
:103142003EAE4BE4FCFDE554254CF554E5533EF50B
:1031520053ED3552F552EC3551F551AF50AE4FADFE
:103162004EAC4DAB54AA53A952A851D312271D40BD
:10317200099080027410F07F002290802CE551F0BB
:10318200A3E552F0A3E553F0A3E554F09080027456
:0431920040F0AF4A10
:013196002216
:103197009081E3E0F54A054A054A054A054A054A8A
:1031A700054A054A054A054A054A90801CE0F54D3F
:1031B700A3E0F54EA3E0F54FA3E0F5509081E4E0DE
:1031C700F54A054A054A054A054A054A054A054A90
:1031D700054A054A054A908020E0F551A3E0F552DB
:1031E700A3E0F553A3E0F554E4F54AE553B54F0AD8
:1031F700E554B55005C2090232E2E553540744E8E5
:10320700F58385548263A20190600463A2017F0E57
:10321700122E54906004E0F54BA3E0F54C90600C3F
:10322700E0FFF4604590667DE0FEEF6E706EA3E010
:10323700FF90600DE06F706490667FE0FF90600E16
:10324700E06F7058906680E0FF90600FE06F704C01
:10325700906681E0FF906010E06F7040906682E0BA
:10326700FF906011E06F60048032D2D9906004E073
:10327700702AA3E024F2F54AE553540744E8F5839E
:10328700855482740E2582F582E43583F58363A223
:103297000190600463A201AF4A122E54AE4BE4FCC6
:1032A700FDE554254CF554E5533EF553ED3552F500
:1032B70052EC3551F551AF50AE4FAD4EAC4DAB540E
:1032C700AA53A952A851D312271D5006E54C454BC6
:1032D70070099080017410F07F0022908020E551E2
:1032E700F0A3E552F0A3E553F0A3E554F090800175
:0532F7007440F0AF4A35
:0132FC0022AF
:043726008E4F8F50E3
:10372A00906C4FE0FCA3E0FDA3E0FEA3E0F5568E0B
:10373A00558D548C53E556FFE5555407FEE42FF595
:10374A0052EE34C0F551855282F5837423F0055246
:10375A00E552700205515351C7F582855183740AA7
:10376A00F00552E552700205515351C79063416307
:10377A00A20185518385528263A2017F06122E100F
:10378A0074062552F552E43551F551854F8385501B
:10379A008263A20185518385528263A201122DF4AC
:1037AA00908000E020E5F9E4FCFDFE906C4FE0F823
:1037BA00A3E0F9A3E0FAA3E02FFFEE3AFEED39FD0C
:1037CA00EC38FCEF2408FFE43EFEE43DFDE43CFC5B
:1037DA00906C4F122741906C4FE0908040F0906CB3
:1037EA0050E0908041F0906C51E0908042F0906CF3
:0C37FA0052E0908043F09080007420F0BA
:01380600229F
:0638E1008E4F8F508D5147
:1038E700906C4FE0FCA3E0FDA3E0FEA3E0F5578E4C
:1038F700568D558C54E557FFE5565407FEE42FF5D2
:1039070053EE34C0F552855382F5837423F0055383
:10391700E553700205525352C7F582855283EBF087
:103927000553E553700205525352C790634163A292
:103937000185528385538263A2017F06122E10747C
:10394700062553F553E43552F552854F838550824A
:1039570063A20185528385538263A201AF51122E60
:1039670010908000E020E5F974082551F551FFE437
:10397700FCFDFEE5572FF557EE3556F556ED355557
:10398700F555EC3554F554908040E554F0A3E555D2
:10399700F0A3E556F0A3E557F09080007420F0AF50
:0D39A70057AE56AD55AC54906C4F122741F1
:0139B40022F0
:023E27008F63A7
:103E2900906C4FE0FCA3E0FDA3E0FEA3E0F5678EF4
:103E3900668D658C64E567FFE5665407FEE42FFF30
:103E4900EE34C09062B763A201F5838F8263A20149
:103E5900AF63122E10908000E020E5F9E4FCFDFE2E
:103E6900E5672563F567EE3566F566ED3565F56554
:103E7900EC3564F564908040E564F0A3E565F0A352
:103E8900E566F0A3E567F09080007420F0AF67AEB7
:0B3E990066AD65AC64906C4F122741D1
:013EA40022FB
:063807008E4F8F50AB054F
:10380D00906C4FE0FCA3E0FDA3E0FEA3E0F5568E27
:10381D00558D548C53E556FFE5555407FEE42FF5B1
:10382D0052EE34C0F551855282F5837423F0055262
:10383D00E552700205515351C7F582855183EBF066
:10384D000552E5527002055190634163A201855105
:10385D008385528263A2017F06122E1074062552B3
:10386D00F552E43551F5515351C7E54F85528285D7
:10387D005183F00552E552700205515351C7F5823F
:10388D00855183E550F00552E552700205515351B3
:10389D00C7908000E020E5F9E556240AF556E43599
:1038AD0055F555E43554F554E43553F553908040B2
:1038BD00E553F0A3E554F0A3E555F0A3E556F090DC
:1038CD0080007420F0AF56AE55AD54AC53906C4F94
:0338DD001227416E
:0138E00022C5
:1044D200E5D220E0FBC2AF438E2075D2028F828EDE
:0B44E20083E0FFE4F5D2538EDFD2AF81
:0144ED0022AC
:10450800E5D220E0FBC2AF43D2028F828E83EDF06A
:0945180075D25063D250D2AF22DB
:103EA500E4FDED2401FFE433FE1244D274392DF50F
:103EB50082E43463F583EFF00DBD3FE6E4FDED24C8
:103EC5007FFFE433FE1244D2742F2DF582E4346172
:103ED500F583EFF0742F2DF582E43461F583E070FE
:103EE5001B742F2DF582E43461F5837420F0743052
:103EF5002DF582E43461F583E4F080040DBD80BEC8
:103F0500E49061AEF0FDEDFF7E001244D274AF2D5A
:0D3F1500F582E43461F583EFF00DBDFEE9A7
:013F2200227C
:024413008B4FCD
:10441500A2AF920FC2AF85A25053A2FE8E838F82A8
:1044250005A28C838D827409122E6CE54F53A2FE72
:1044350043A220122E6E53A2DF8550A2A20F92AF87
:01444500FF77
:014446002253
:1044B500A2AF920FC2AF8C838D82EF122E6C43A2F6
:0C44C50020122E6E53A2DFA20F92AFFF58
:0144D10022C8
:02446D008F4A74
:10446F00A2AF920FC2AFE4F5838D827406122E6C49
:10447F00E54A43A220122E6E53A2DFA20F92AF7F06
:01448F00012B
:014490002209
:024491008F4A50
:10449300A2AF920FC2AFE4F5838D82740A122E6C21
:1044A300E54A43A220122E6E53A2DFA20F92AF7FE2
:0144B3000107
:0144B40022E5
:102CCC00A907E7FFA805EF93C3966008403B74FC87
:102CDC002FFF80F00F08EF93C3966008402B74FB16
:102CEC002FFF80E00F08EF93C3966008401B74FA27
:102CFC002FFF80D00F08EF93D3966008400B74F928
:102D0C002FFF80C01F1F1F1F1FEF54FEF80303F778
:102D1C00E893FC08E893FD08E893FE08E893FF228B
:102D2C0009E993C39D6008402974FB29F980F109D6
:102D3C00E993C39E6008401A74FA29F980E209E904
:102D4C0093D39F6008400B74F929F980D319191992
:102D5C001919E9C313C313FF22740093F8ECC39839
:102D6C004024701F740193F8EDC3984019701474CB
:0E2D7C000293F8EEC398400E7009740393F8AA
:102D8A00EFC39840037F00227F0122EDF8E6F008A6
:102D9A00A3DFFA22EDF8E0F608A3DFFA22E0A36344
:102DAA00A201F0A363A201DFF475A20022E0A363EB
:102DBA00A201F0A363A201E0A363A201F0A363A2AC
:102DCA0001E463A201F0A363A201DFE175A200227C
:102DDA00E0A363A2016DFE936CFDEE058393FC15DF
:102DEA008363A201DFEA75A200227F00E493A36352
:102DFA00A201F00F600CA3E583C2E3F58363A2018D
:102E0A0080EA75A20022E0A363A201F0A3E583C2CF
:102E1A00E3F58363A201DFEE75A20022E0A363A2B9
:102E2A0001F0A3E583C2E4D2E3F58363A201DFECF8
:102E3A0075A20022E583C2E3F583E0A363A201F051
:102E4A00A363A201DFEE75A20022E583C2E4D2E306
:102E5A00F583E0A363A201F0A363A201DFEC75A2EC
:102E6A000022F922C002C004C00612FFF0D006D028
:042E7A0004D002225C
:101E21003E2A2C312CCFE0F0E0ECE5F2F0FB20F87B
:101E3100E8EDFB2043414E0A003E4C2C6B30312C27
:101E410025732C43EAEEF0EEF1F2FC20EDE020F8F0
:101E5100E8EDE52043414E2C30202D20353030EA8D
:101E6100E1283530EC292C31202D203530EAE128CC
:101E7100353030EC290A0030202D20353030EAE1B0
:101E8100283530EC290031202D203530EAE1283584
:101E91003030EC29003E2A2C312CCFE0F0E0ECE58B
:101EA100F2F0FB20EFF0EEF2EEEAEEEBE020D1DD16
:101EB100D22D34D2CC0A003E4C2C4930312C256C29
:101EC100752CD1EAEEF0EEF1F2FC20EEE1ECE5ED5D
:101ED100E02C313230302C323430302C3438303048
:101EE1002C393630302C31393230300A003E532C07
:101EF1004931322C2562752CC0E4F0E5F120E1EB8B
:101F0100EEEAE020D2C8D220EDE020F8E8EDE50AC3
:101F1100003E532C6D2562752C25732CCFF0E8E122
:101F2100EEF0202562752028C0E4F0E5F120E820DC
:101F3100EFE0F0E0ECE5F2F0FB290A003E532C560D
:101F410030382C2562752CC8EDF2E5F0E2E0EB208B
:101F5100EEEFF0EEF1E0282A3130ECF1290A003CF5
:101F610021003C6B30313D003C4930313D003C4962
:101F710031323D003C5630383D002043616E4572A0
:101F810047495400200A002043616E45727243485C
:101F910021000A000ACEF2EAF0FBF2FC3A000A46FE
:101FA10069783A000AC7E0EFF0EEF13A00CFF0E8C5
:101FB100E5EC3A00CEF8E8E1EAE020CAD1210A00D6
:101FC100CED8C8C1CAC020C0E4F0E5F1E02100CEFE
:101FD100D8C8C1CAC020EEF2EAF0FBF2E8FF20EA5D
:101FE100E0EDE0EBE02100204F4B212000CED8C8EE
:101FF100C1CAC020E7E0EFF0EEF1E00000C181408E
:1020010001C0804101C0804100C1814001C08041C7
:1020110000C1814000C1814001C0804101C08041B7
:1020210000C1814000C1814001C0804100C18140A7
:1020310001C0804101C0804100C1814001C0804197
:1020410000C1814000C1814001C0804100C1814087
:1020510001C0804101C0804100C1814000C1814077
:1020610001C0804101C0804100C1814001C0804167
:1020710000C1814000C1814001C0804101C0804157
:1020810000C1814000C1814001C0804100C1814047
:1020910001C0804101C0804100C1814000C1814037
:1020A10001C0804101C0804100C1814001C0804127
:1020B10000C1814000C1814001C0804100C1814017
:1020C10001C0804101C0804100C1814001C0804107
:1020D10000C1814000C1814001C0804101C08041F7
:1020E10000C1814000C1814001C0804100C18140E7
:1020F10001C0804101C0804100C1814000C0C101D7
:10210100C30302C2C60607C705C5C404CC0C0DCD66
:102111000FCFCE0E0ACACB0BC90908C8D81819D9D6
:102121001BDBDA1A1EDEDF1FDD1D1CDC14D4D51506
:10213100D71716D6D21213D311D1D010F03031F1F6
:1021410033F3F23236F6F737F53534F43CFCFD3D26
:10215100FF3F3EFEFA3A3BFB39F9F83828E8E92916
:10216100EB2B2AEAEE2E2FEF2DEDEC2CE42425E5C6
:1021710027E7E62622E2E323E12120E0A06061A136
:1021810063A3A26266A6A767A56564A46CACAD6DE6
:10219100AF6F6EAEAA6A6BAB69A9A86878B8B97956
:1021A100BB7B7ABABE7E7FBF7DBDBC7CB47475B586
:1021B10077B7B67672B2B373B17170B05090915176
:1021C1009353529296565797559594549C5C5D9DA6
:1021D1005F9F9E5E5A9A9B5B995958988848498996
:1021E1004B8B8A4A4E8E8F4F8D4D4C8C4484854546
:1021F1008747468682424383418180403C6D303D22
:10220100000000003C6D313D000000003C6D323D9E
:10221100000000003C6D333D000000003C6D343D8A
:10222100000000003C6D353D000000003C6D363D76
:10223100000000003C6D373D000000003C6D383D62
:10224100000000003C6D393D000000003C6D313064
:102251003D0000003C6D31313D0000003C6D3132EC
:102261003D0000003C6D31333D0000003C6D3134D8
:0C2271003D0000003C6D31353D000000D8
:0100210022BC
:0300230002409206
:0B409200C0E0C083C082C0D075D01811
:10409D00309827E5E92464F5EB30D707E5F904F509
:1040AD00FB800385F9FBD291742B2537F582E4341F
:1040BD006BF583E599F00537C298309931E53CC32E
:1040CD009536501BAF3C053C742B2FF582E4346CB8
:1040DD00F583E0FF521FA2D0B3929B8F99800DE51F
:0E40ED003CC395364006053CD296C290C2995F
:0940FB00D0D0D082D083D0E03295
:1032FD007BFF7A1E79211222DF90688FE0701475A2
:10330D0052FF75531E7554787BFF7A1E793A12223F
:10331D00DF80127552FF75531E7554877BFF7A1E21
:10332D00793A1222DF7BFF7A1E79961222DF906C9A
:10333D004DE0FEA3E0FFC3E49FFFE49EFEAB07FA62
:10334D003395E0F9F87F007E8C7D0A7C0012267D96
:10335D008F558E548D538C527BFF7A1E79B8122265
:10336D00DF7BFF7A1E79EE906890E0F5521222DF36
:10337D00E4906C5BF0906C5BE0FFC36480949040D4
:10338D000302341F906A9A7420F0E4A3F0EF339592
:10339D00E0FEEF7803C333CE33CED8F924FDF582AA
:1033AD0074213EAF82FE123C9CEF4E6041E4906C66
:1033BD005DF01244EE906C5CEFF0643C601BE0FF3E
:1033CD00A3E0FE04F0EEFD3395E0FC749A2DF5823A
:1033DD00746A3CF583EFF080D9906C5DE0FF339516
:1033ED00E0FE749A2FF582746A3EF583E4F0906CDA
:1033FD005BE0F55275530175546A75559A04F5568F
:10340D007BFF7A1F79121222DF906C5BE004F002D1
:10341D0033827BFF7A1F793D906C4CE0F55212227E
:01342D00DFBF
:01342E00227B
:06439700AC05AB07AA060D
:10439D00906A9974FFF0906AEAF0AF041CEF602DFB
:1043AD000BEBAE0270010A14F5828E83E0FF906A6A
:1043BD0099E06FFF901FFD93FE906AEAE06E906AA0
:0D43CD0099F0EF9020FD93906AEAF080CD0A
:0143DA0022C0
:04410400A907AE0356
:10410800E4906C5BF0906C5BE0FFC394405014E566
:10411800422FF582E43541F583E4F0906C5BE004CE
:10412800F080E2854282854183E9F0A37408F0EECD
:10413800D39401400D854282854183A3A37416F070
:10414800800B854282854183A3A37414F085428243
:10415800854183A3A3A3EDF0E542240CF582E43561
:0541680041F583EEF0BB
:01416D00222F
:100E9E007E1F7F60123C9CEF4E70037F0122E49018
:100EAE00688FF07E1F7F63123C9CEF4E601B1244D6
:100EBE00EE8F4AE54AB4310690688F740AF0E54A1F
:100ECE00B4320690688F7464F07E1F7F69123C9C6A
:100EDE00EF4E602312429AA804A905AA06AB077F1B
:100EEE00007E8C7D0A7C0012267D12270F906C4DA1
:100EFE00EEF0A3EFF0800A906C4D74FFF0A374B87F
:100F0E00F07E1F7F6F123C9CEF4E600A12429A9049
:100F1E006890EFF08005E4906890F07E1F7F751268
:100F2E003C9CEF4E600D12429A906C4BEEF0A3EF8C
:100F3E00F08009906C4BE4F0A37464F0E4F541F595
:100F4E004285428285418374FEF0A37403F085428C
:100F5E0082854183A3A37408F0854282854183A3D1
:100F6E00A3A37455F0E5422404F582E43541F583DC
:100F7E0074AAF0E5422405F582E43541F583743315
:100F8E00F0E5422406F582E43541F58374CCF07D1C
:100F9E0007AF42AE41124397906A99E0FFE54224B3
:100FAE0007F582E43541F583EFF0906AEAE0FFE55C
:100FBE00422408F582E43541F583EFF074102542A2
:100FCE00F542E43541F541854282F583E4F0906ABD
:100FDE009804F0E4F54AAF4AEF3395E0FEEF78035C
:100FEE00C333CE33CED8F924FDF58274213EAF82C1
:100FFE00FE123C9CEF4E700302139812429A8F43DE
:10100E00E54370030213A6854282854183E543F0D2
:10101E00A37401F0854282854183A3A37430F085C9
:10102E004282854183A3A3A3F0E5422404F582E422
:10103E003541F5837430F0E5422405F582E43541FF
:10104E00F5837430F0E5422406F582E43541F583EC
:10105E007430F0E5422407F582E43541F5837430AF
:10106E00F07D08AF42AE41124397906A99E0FFE5DA
:10107E00422408F582E43541F583EFF0906AEAE008
:10108E00FFE5422409F582E43541F583EFF0E542B0
:10109E00240CF582E43541F583E4F074102542F515
:1010AE0042E43541F541906A98E004F0854282852C
:1010BE004183E4F01244EEEF12277E11A40011A436
:1010CE0021110F2313862A135D2F112E3B11A43CE1
:1010DE00135D3E127743128345124746126B491237
:1010EE005F4C122350122F51137452123B53125352
:1010FE005512E261130B6213346312BB73000010BE
:10110E00C21244EE75F008EFA42475F582E5F034B2
:10111E0020AF82FE123C9CEF4E609912429A809450
:10112E007D04AF42AE41124397906A99E0FFE542CB
:10113E002404F582E43541F583EFF0906AEAE0FF8E
:10114E00E5422405F582E43541F583EFF07D06AFE7
:10115E0042AE41124397906A99E0FFE5422406F5AC
:10116E0082E43541F583EFF0906AEAE0FFE5422430
:10117E0007F582E43541F583EFF074102542F54210
:10118E00E43541F541906A98E004F085428285414C
:10119E0083E4F00210C2854282854183E0606B7D5C
:1011AE0004AF42AE41124397906A99E0FFE54224A4
:1011BE0004F582E43541F583EFF0906AEAE0FFE54D
:1011CE00422405F582E43541F583EFF07D06AF420A
:1011DE00AE41124397906A99E0FFE5422406F582EC
:1011EE00E43541F583EFF0906AEAE0FFE54224072B
:1011FE00F582E43541F583EFF074102542F542E4B3
:10120E003541F541906A98E004F08542828541832C
:10121E00E4F00213987B0FE4FDAF43124104021079
:10122E00C27B0F7D04AF431241040210C27B0F7DBF
:10123E0008AF431241040210C27B017D40AF43123E
:10124E0041040210C27B0E7D10AF43124104021006
:10125E00C27B0E7D14AF431241040210C27B0E7D81
:10126E0020AF431241040210C27B0F7D30AF4312F8
:10127E0041040210C27B017D0FAF4312410485422F
:10128E0082854183A37405F0854282854183A3A3A1
:10129E00E4F0854282854183A3A3A3F0E542240CAA
:1012AE00F582E43541F5837401F00210C285428265
:1012BE00854183A3A37411F0854282854183A3A344
:1012CE00A3E0F0E542240CF582E43541F583740188
:1012DE00F00210C2854282854183A3A37411F0856A
:1012EE004282854183A3A3A3E04401F0E542240C8E
:1012FE00F582E43541F5837401F00210C285428215
:10130E00854183A3A37411F0854282854183A3A3F3
:10131E00A3E04402F0E542240CF582E43541F58366
:10132E007401F00210C2854282854183A3A3741119
:10133E00F0854282854183A3A3A3E04403F0E542F6
:10134E00240CF582E43541F5837401F00210C212CB
:10135E0044EEEF24D0FFE542240DF582E43541F54D
:10136E0083EFF00210C2E542240EF582E43541F51A
:10137E0083E04401F00210C2E542240EF582E4350A
:10138E0041F583E04402F00210C2054AC3E54A6407
:10139E008094905003020FE4E4F541F542F54A853E
:1013AE004282854183E06073A3E064087034E542B5
:1013BE00240FF582E43541F583E54AF0E542240C2D
:1013CE00F582E43541F583E0FFB40102054AEFB43E
:1013DE000F067404254AF54AEFB40E067403254A27
:1013EE00F54A854282854183A3E0B40521E5422476
:1013FE000FF582E43541F583E54AF0E542240CF51C
:10140E0082E43541F583E0B40104054A054A7410BF
:10141E002542F542E43541F5418084E4F541F5423B
:01142E00FFBE
:01142F00229A
:10444700C2A9438902758C48758A4875D90475DBFA
:104457004875DC4875DD4875DE48E4F5E9F5F9C2CD
:06446700D9D28CD2DE2246
:10416E0043AB01C2E8C2EAE4FFEFC454F0F5B1C3B9
:10417E00EF64809488500575B3D08003E4F5B3E402
:10418E00F5B275BCC8F5BDF5BE75BF7875C4FFF543
:10419E00C5F5C675C778F5A3F5A3F5A3F5A3F5A3E5
:1041AE00F5A3F5A3F5A30FBF0EBF90688FE0FF2513
:1041BE00E0F5B475B50C75B66C75A11275AB0275DC
:0841CE00C13E75C3FF75C20379
:0141D60022C6
:10423A0075B180E4F5B3F5B28526BCE5275403FFD2
:10424A0033333354F8FFE52754E04FFFE528C4130E
:10425A0054074FF5BDE52833333354F8FFE529C435
:10426A001354074FF5BEE52933333354F8F5BF85A8
:10427A002BA3852CA3852DA3852EA3852FA385305B
:10428A00A38531A38532A3E52A540F2450F5B3221E
:10342F00E59B541F6020200A1A7E1F7F7B123726D0
:10343F00E59B541FFF7E007D031238077E1F7F859B
:10344F00123726E4F59BE5BA30E008E4F5B375B121
:10345F0080F5B2E5CFF47003023539754C01E4F510
:10346F004BE5CFF4554C7003023527E54BC454F0B0
:10347F00F5B1E5B2547F6420706FE5B3540FF52AB0
:10348F0085BC26E5BD541FFF131313541FFFE5BD65
:10349F0054E044184FF527E5BDC43354E0FFE5BEB3
:1034AF00131313541F4FF528E5BEC43354E0FFE543
:1034BF00BF131313541F4FF52985A32B85A32C85F9
:1034CF00A32D85A32E85A32F85A33085A33185A397
:1034DF0032E4F5B2E526547EB5260575B350800368
:1034EF0075B3D0E52A2405FF22E5B2549F6023204F
:1034FF000A207E1F7F88123726AFB27E007D03120F
:10350F003807AFB37E007D031238077E1F7F9312FB
:10351F003726E4F5B275B3D0E54C25E0F54C054BF5
:0C352F00E54BC3940850030234707F0089
:01353B00226D
:103C1500C218E4F537F50BD296F536F53CF524FFD9
:103C25007F40906AEBE4F0A3DFFC7F40E4906A9666
:103C3500F0A3F0F53DF548120E9E12416EC2ADE4BB
:103C4500F5C9D2CDD2CCC2C9C2CAF5CDF5CC906CDE
:103C55004DE0F5CBA3E0F5CA85CBCD85CACCE4F51F
:103C6500985387BFD29FD29E438740C29FC2ACC2A2
:103C750098C29975B81075B710D2CAD29CD2AC1239
:103C85004447C2D9E5E92464F5EB30D706E5F904E4
:063C9500F5FB2285F9FB9E
:013C9B002206
:0100220022BB
:01453C00225C
:01453D00225B
:01453E00225A
:10287F00854282854183E0F5437012F541F542852B
:10288F004282854183E0F54370037F0122854282B6
:10289F00854183A3E0FE640160030229757533014E
:1028AF00854134854235E542240CF582E43541F506
:1028BF0083E0601674102542F542E43541F54185F9
:1028CF004282F583E070A97F012285428285418390
:1028DF00E0906C2BF0A3EEF0854282854183A3A399
:1028EF00E0906C2DF0854282854183A3A3A3E090F5
:1028FF006C2EF0E5422404F582E43541F583E09037
:10290F006C2FF0E5422405F582E43541F583E09024
:10291F006C30F0E5422406F582E43541F583E09012
:10292F006C31F0E5422407F582E43541F583E09000
:10293F006C32F0E5422408F582E43541F583E090EE
:10294F006C33F0E5422409F582E43541F583E090DC
:10295F006C34F075360A300A03022AB87E1F7F9551
:10296F00123726022AB8854282854183A3E0FF648D
:10297F00036003022A1C052453240F906A96F0A3C8
:10298F00F0854282854183E0906C2BF0A3EFF085B8
:10299F004282854183A3A3E0906C2DF0854282850E
:1029AF004183A3A3A3E0906C2EF0E5422404F582AB
:1029BF00E43541F583E0906C2FF0E5422405F58274
:1029CF00E43541F583E0906C30F0E5422406F58262
:1029DF00E43541F583E0906C31F0E5422407F58250
:1029EF00E43541F583E0906C32F0E5422408F5823E
:1029FF00E43541F583E0906C33F0753609300A0306
:102A0F00022AB87E1F7F9F123726022AB8AB33AA3D
:102A1F0034A93590000C1225F2700E74102542F572
:102A2F0042E43541F54102287FE542240EF582E468
:102A3F003541F583E030E112E524600E7410254234
:102A4F00F542E43541F54102287F85428285418375
:102A5F00E0906C2BF0854282854183A3E0906C2C33
:102A6F00F0854282854183A3A3E0906C2DF08542CF
:102A7F0082854183A3A3A3E0906C2EF0E54224044A
:102A8F00F582E43541F583E0906C2FF0E5422405A3
:102A9F00F582E43541F583E0906C30F07536062011
:102AAF000A077E1F7FA5123726E4F53CD290C2910C
:102ABF00C296C2992099FDD299200A0B7E6C7F2B6A
:092ACF00E4FBAD361238E17F0092
:012AD80022DB
:103AFB00E548C394404003E4F54874EB2548F58250
:103B0B00E4346AF583E0FF30E16F74EB2548F5820E
:103B1B00E4346AF583EF54FDF0E4906478F0A37419
:103B2B000DF090667CE090647AF0A37419F0A374A6
:103B3B0048F0A37479F0E548131313541FFF9068F2
:103B4B0090E02F90647EF0E548540725E025E024B3
:103B5B0080A3F0A37408F0F5F0E548A4248FF58258
:103B6B00E5F03466F58363A20190648163A2017F63
:0E3B7B0008122DA705487F012205487F002271
:01453F002259
:10197A0074EB253DF582E4346AF583E020E0020544
:10198A003DE53DC394404003E4F53D12342FEF603A
:10199A0069E529640F7063906890E0FF6528705AC2
:1019AA0074EB253DF582E4346AF583E0FE30E04AC3
:1019BA0074EB253DF582E4346AF583EE54FEF07546
:1019CA002648752779E53D131313541FFEEF2EF5AC
:1019DA0028E53D540725E025E02480F529752A08E5
:1019EA0075F008E53DA4248FF582E5F03466F583A9
:1019FA007D2B7F08122D9E12423A300249C2029074
:101A0A006892E004F07006906891E004F0D3906860
:101A1A0092E094B8906891E0940B402AE4F0A3F025
:101A2A00F54A74EB254AF582E4346AF583E030E23C
:101A3A000E74EB254AF582E4346AF5837403F005E3
:101A4A004AE54AB440DC20D903021E20C2D9E53750
:101A5A00D394005003021DD4C291853740E4F53770
:101A6A00F50B7E6B7F2BAD40124397200A127E1F27
:101A7A007FAE1237267E6B7F2BE4FBAD401238E136
:101A8A00906AEAE0FF906A99E04F6010300A030218
:101A9A001DD47E1F7FB5123726021DD4906B2BE012
:101AAA0065436010300A03021DD47E1F7FC11237BE
:101ABA0026021DD4854282854183A3E06401703DDC
:101ACA00906B2CE0601A200A077E1F7FD0123726FF
:101ADA00E542240CF582E43541F583E4F0021DD495
:101AEA00D219200A077E1F7FE8123726E542240C06
:101AFA00F582E43541F5837401F0021DD4D219E56B
:101B0A0040C39406501DAB33AA34A93590000CE4A7
:101B1A0012261F300A03021DD47E1F7FEE123726BB
:101B2A00021DD4E542240FF582E43541F583E075C0
:101B3A00F002A4FF906A96E5F0F0A3EFF0E4F54A0C
:101B4A00E542240CF582E43541F583E0FD7C00741E
:101B5A00017E00A84A088005C333CE33CED8F9FFE8
:101B6A00EE5CFEEF5D4E7003021DC985428285411F
:101B7A0083A3E064086003021CAFF538E54A75F0F8
:101B8A0003A4242CF582E4346BF583E0543FF53941
:101B9A00E54A75F003A4242DF582E4346BF583E05D
:101BAA00F53AE54A75F003A4242EF582E4346BF580
:101BBA0083E0F53BAF3BAE3AAD39AC38E542240D94
:101BCA00F582E43541F583E0F9F812272E8F3B8E32
:101BDA003A8D398C38E542240EF582E43541F58395
:101BEA00E030E026E54A75F003A4242CF582E434BB
:101BFA006BF583E030E713AF3BAE3AAD39AC381240
:101C0A00270F8F3B8E3A8D398C38906A96E0FEA367
:101C1A00E0248FF58274663EF583E0653B60299087
:101C2A006A96E0A3E0FF248FF58274663EF583E5A9
:101C3A003BF0EF7803CEC313CE13D8F924EBF58229
:101C4A00746A3EF5837407F0906A97E004F07006B0
:101C5A00906A96E004F0906A96E0FEA3E0248FF57D
:101C6A008274663EF583E0653A6029906A96E0A33D
:101C7A00E0FF248FF58274663EF583E53AF0EF784B
:101C8A0003CEC313CE13D8F924EBF582746A3EF55A
:101C9A00837407F0906A97E004F07006906A96E001
:101CAA0004F0021DC9E54A75F003A4242FF582E465
:101CBA00346BF583E0FF906A96E0FCA3E0FD248F85
:101CCA00F58274663CF583EFF0EDAE047803CEC37B
:101CDA0013CE13D8F924EBF582746A3EF5837404A3
:101CEA00F0906A97E004F07006906A96E004F0E5D6
:101CFA004A75F003A4242EF582E4346BF583E0FFE1
:101D0A00906A96E0FCA3E0FD248FF58274663CF5A8
:101D1A0083EFF0EDAE047803CEC313CE13D8F924C3
:101D2A00EBF582746A3EF5837404F0906A97E004D6
:101D3A00F07006906A96E004F0E54A75F003A42470
:101D4A002DF582E4346BF583E0FF906A96E0FCA3FC
:101D5A00E0FD248FF58274663CF583EFF0EDAE0466
:101D6A007803CEC313CE13D8F924EBF582746A3EF6
:101D7A00F5837404F0906A97E004F07006906A960E
:101D8A00E004F0E54A75F003A4242CF582E4346BF0
:101D9A00F583E0FF906A96E0FCA3E0FD248FF582CC
:101DAA0074663CF583EFF0EDAE047803CEC313CE30
:101DBA0013D8F924EBF582746A3EF5837404F005AE
:101DCA004AE54A64046003021B4A20190DAB33AA90
:101DDA0034A93590000CE412261FE536600B741006
:101DEA002542F542E43541F541E5E924E8F5EB30D1
:101DFA00D708E5F92404F5FB8006E5F92403F5FB89
:101E0A0012287FEF7010854282854183A3E0B403D4
:061E1A0003D21922C219D7
:011E2000229F
:03001E007F00223E
:103B9500020881E493A3F8E493A34003F68001F2BD
:103BA50008DFF48029E493A3F85407240CC8C33331
:103BB500C4540F4420C8834004F456800146F6DF00
:103BC500E4800B0102040810204080904535E47E16
:103BD500019360BCA3FF543F30E509541FFEE493F5
:103BE500A360010ECF54C025E060A840B8E493A3BC
:103BF500FAE493A3F8E493A3C8C582C8CAC583CAE7
:103C0500F0A3C8C582C8CAC583CADFE9DEE780BE9E
:01453B00007F
:1025D900BB010689828A83E0225002E722BBFE0200
:0925E900E32289828A83E4932233
:1025F200BB010CE58229F582E5833AF583E022509E
:1026020006E92582F8E622BBFE06E92582F8E222E7
:0D261200E58229F582E5833AF583E4932201
:10261F00F8BB010DE58229F582E5833AF583E8F0F1
:10262F00225006E92582C8F622BBFE05E92582C89D
:02263F00F22285
:1026410075F008758200EF2FFFEE33FECD33CDCC50
:1026510033CCC58233C5829BED9AEC99E5829840D3
:102661000CF582EE9BFEED9AFDEC99FC0FD5F0D6B0
:10267100E4CEFBE4CDFAE4CCF9A88222B800C1B9DA
:102681000059BA002DEC8BF084CFCECDFCE5F0CB18
:10269100F97818EF2FFFEE33FEED33FDEC33FCEB51
:1026A10033FB10D703994004EB99FB0FD8E5E4F90C
:1026B100FA227818EF2FFFEE33FEED33FDEC33FCF9
:1026C100C933C910D7059BE99A4007EC9BFCE99AED
:1026D100F90FD8E0E4C9FAE4CCFB2275F010EF2F32
:1026E100FFEE33FEED33FDCC33CCC833C810D70732
:1026F1009BEC9AE899400AED9BFDEC9AFCE899F86D
:0E2701000FD5F0DAE4CDFBE4CCFAE4C8F922FF
:0E270F00C3E49FFFE49EFEE49DFDE49CFC22DB
:10271D00EB9FF5F0EA9E42F0E99D42F0E89C45F012
:01272D002289
:10272E00E8600FECC313FCED13FDEE13FEEF13FF89
:03273E00D8F122AD
:0C274100ECF0A3EDF0A3EEF0A3EFF0220B
:10274D00A8828583F0D083D0821227641227641269
:10275D002764122764E473E493A3C583C5F0C5838E
:10276D00C8C582C8F0A3C583C5F0C583C8C582C8D6
:01277D002239
:10277E00D083D082F8E4937012740193700DA3A3EA
:10278E0093F8740193F5828883E4737402936860FE
:06279E00EFA3A3A380DFFE
:10227D00E55E2452F8E6055E22784F30160278525C
:10228D00E475F0011228050225D9200FEB7F2ED21F
:10229D000F8018EF540F2490D43440D4FF30130B1B
:1022AD00EF24BFB41A0050032461FFE55F600215EF
:1022BD005F0562E5627002056130160D784FE475B9
:1022CD00F001122805EF0227A40243507403D21621
:1022DD008003E4C216F55E8B4F8A508951E4F55F99
:1022ED00F561F562E55F60077F201222B880F57514
:1022FD0060FFC210C20FC211C212C214C215C217A2
:10230D00122286FF700D3016057F001222C9AF62B2
:10231D00AE6122B4255FC2D5C213122286FF24D02E
:10232D00B40A00501A75F00A785F30D50508B6FF6B
:10233D000106C6A426F620D5047002D21280D92437
:10234D00CFB41A00EF5004C2E5D2130224C9D21043
:10235D0080C6D20F80C0D21180BCD2D580BAD21423
:10236D0080B47F201222B82011077401B55F0040A0
:10237D00F112227DFF1222B80222F1D217D215805E
:10238D009512227DFB12227DFA12227DF94A4B70A5
:10239D0006799A7A257BFF20112EE55F602A7E0053
:1023AD008E827583001225F260060EEE656070F068
:1023BD00C2D5EBC0E0EAC0E0E9C0E0EE122510D0D6
:1023CD00E0F9D0E0FAD0E0FB1225D9FF60AAEBC00E
:1023DD00E0EAC0E0E9C0E01222B8D0E02401F9D073
:1023ED00E03400FAD0E0FBE5600460DCD560D98014
:1023FD00877BFF7A25790CD211809C791080027928
:10240D0008C215C2178008D2D5790A8004790AC28C
:10241D00D5E560047002F560E4FAFDFEFF12227D41
:10242D00FC7B0820101312227DFD7B10300F0A1249
:10243D00227DFE12227DFF7B20EC3382D592D5507A
:10244D0013C3E4300F069FFFE49EFEE42010039DAE
:10245D00FDE49CFCE4CBF8C210EC700CCFCECDCCDF
:10246D00E824F8F870F38017C3EF33FFEE33FEED79
:10247D0033FDEC33FCEB33FB994002FB0FD8E9EB5A
:10248D00301005F8D0E0C448B210C0E00AEC4D4E53
:10249D004F78207B0070C2EAB5600040BCC0E012EE
:1024AD002512D0F0D0E0201004C4C0E0C4B210C09A
:1024BD00F01222A1D0F0D5F0EB0222F112277E23EB
:1024CD008E53240858235F4C235B42240C4F241455
:0F24DD0044241449237443241A5523FE4623FE36
:1024EC004523FE4725BA5023632D23672E238A2BC1
:1024FC00236B2323882025A32A232348000023822F
:10250C003F3F3F00790AA2D5201214301409B910AC
:10251C00020404B9080104A2D520150250010420BC
:10252C0011689211B55F005034C0E07F2030121951
:10253C007F30A21172157214500F122569C211C28C
:10254C0015C214C2177F30800F301403E9C0E0129B
:10255C0022B8301403D0E0F9D0E0B55FCC301417BA
:10256C007F30B9100C1222B87F583013077F788057
:10257C0003B908031222B83011057F2D0222B87F4F
:10258C00202017F87F2B2015F322921180CF286E74
:10259C00756C6C2900D21012227D3010F8C21078A4
:1025AC005F30D50108F60223232D504349581222DF
:1025BC007D2403B405004001E49025B5931222A9B3
:0D25CC00743A1222A9D212755F040224088D
:102E7E008B4F8A508951E4F55BF55AF559F558F5A3
:102E8E0056F557E553455445526012EBC0E0EAC083
:102E9E00E0E9C0E0AB52AA53A954122815AB4F0576
:102EAE0051E551AA507002055014F91225D9F55C5E
:102EBE00C394094007E55CD3940D40E1E55C6420C2
:102ECE0060DBE55CB42D054357038016E55CB42B3F
:102EDE0005435701800C74FF2551F55174FF355091
:102EEE00F550E55560046410703FAB4FAA50A951E0
:102EFE001225D964306009E555702E75550A802962
:102F0E009000011225F2FF64786004EFB458134369
:102F1E00570175551074022551F551E43550F55091
:102F2E008007E5557003755508AB4F0551E551AA5D
:102F3E00507002055014F91225D9F55CC394614006
:102F4E000AE55CD3947A5003535CDF74D0255CF5AC
:102F5E005CC3940A400CE55C9411406D74F9255CD9
:102F6E00F55CE55CD395555060435701855B6085F4
:102F7E005A5F85595E85585DAF557E00E4FCFDAB0A
:102F8E005BAA5AA959A8581227B6C8ECC8C9EDC9E8
:102F9E00CAEECACBEFCBE4FCFDFEEB255CF55BEE97
:102FAE003AF55AED39F559EC38F558AF5BAE5AADE6
:102FBE0059FCAB60AA5FA95EA85DD312271D500312
:102FCE00022F37435704022F37E55720E003E480E2
:102FDE002DE55345544552601EAB4FE55124FFF984
:102FEE00E55034FFFAEBC0E0EAC0E0E9C0E0AB52D6
:102FFE00AA53A954122815E55730E20774FFFFFEB5
:10300E00FDFC22E557AF5BAE5AAD59AC5830E1032B
:04301E0002270F2254
:1027A400BB010689828A83F0225002F722BBFE0114
:0227B400F3220E
:1027B600E88FF0A4CC8BF0A42CFCE98EF0A42CFCC2
:1027C6008AF0EDA42CFCEA8EF0A4CDA8F08BF0A440
:1027D6002DCC3825F0FDE98FF0A42CCD35F0FCEB9F
:1027E6008EF0A4FEA9F0EB8FF0A4CFC5F02ECD3964
:0F27F600FEE43CFCEAA42DCE35F0FDE43CFC22D1
:10280500FAE6FB0808E6F925F0F618E6CA3AF622D4
:10281500BB011A89828A83D0F0D0E0F8D0E0F9D0E4
:10282500E0FAD0E0FBE8C0E0C0F002286D5016E900
:10283500F8D083D082D0E0F9D0E0FAD0E0FBC082B6
:10284500C083022864BBFE16E9F8D083D082D0E0AD
:0F285500F9D0E0FAD0E0FBC082C08302287622DF
:09286400EBF608EAF608E9F62299
:09286D00EBF0A3EAF0A3E9F0226C
:09287600EBF208EAF208E9F22293
:00000001FF
